:10000000092BFF3FFF3FFF3F0000000000000800FA
:10001000123003138312CB00FF30CA00CB0B112820
:100020001428CA0B11280E28CE30CA00CA0B162875
:1000300000000800293003138312CA00CA0B1E28CF
:1000400000000800031383120C0884000E080D043E
:10005000C0000F08C004C0094008800510088400D3
:1000600012081104C0001308C0041408C004C00919
:1000700040088005AC1F3E28110880042C1F422830
:1000800012088004AC1E4628130880042C1E4A283F
:10009000140880040C0884001508031954280D095D
:1000A000C0004008800556280D0880040F08800411
:1000B00004200F09C000400880050E080D04C00090
:1000C0000F08C004C0094008800510088400120809
:1000D0001104C0001308C0041408C004C00940087B
:1000E0008005AC1D7528110880042C1D7928120884
:1000F0008004AC1C7D28130880042C1C8128140863
:1001000080040C088400150803198B280D09C00011
:10011000400880058D280D0880040F088004042005
:100120000F09C00040088005150803199928082008
:100130009A281A20080003138312AC03AC032C087E
:10014000003C0318A828AC030000000000009F2812
:1001500000000000000000000000080003138312EC
:1001600095012A08AC0022200130950008000313F5
:1001700083122A088400800116088400AB01170846
:10018000003A031DC6288019C328C828801DC62828
:100190001808AC009B201908AC009B202B08031901
:1001A000D12880192B141908AC009B202B080319A7
:1001B000D9288019AB141908AC009B202B0803190F
:1001C000E12880192B151908AC009B202B08031976
:1001D000E9288019AB151908AC009B202B080319DE
:1001E000F12880192B161908AC009B202B08031945
:1001F000F9288019AB161908AC009B202B080319AD
:10020000012980192B171908AC009B202B08031912
:1002100009298019AB171708AB061908AC009B20F9
:10022000801D132917292A088400013080002B081B
:10023000C00008000820082008202208C000013063
:10024000C700400803192829C70D4710FF3F22297E
:10025000470891002308C0000130C100400803197D
:100260003529C10D4110FF3F2F2941089200240874
:10027000C0000130C600400803194229C60D4610CF
:10028000FF3F3C29460893002508C0000130C50007
:10029000400803194F29C50D4510FF3F492945085E
:1002A00094002708C0000130C400400803195C29ED
:1002B000C40D4410FF3F562944088D002808C00093
:1002C0000130C300400803196929C30D4310FF3FE3
:1002D000632943088E002908C0000130C20040088D
:1002E00003197629C20D4210FF3F702942088F0082
:1002F0002108900026088C0021088400410847044A
:10030000C0004608C00445084004C1004109C000BF
:100310004008800584174108C000C00940088005D6
:100320002608840043084404C0004208C004C009F1
:10033000400880058417400880052108840045088E
:100340004604C00040088004260884004208800457
:100350004209C0004008800508200F0880040F09EA
:10036000C0004008800508200F0880040F09C00065
:100370004008800508201008840013088004140930
:10038000C000400880050C0884000F0880040F0995
:10039000C0004008800508200F0880040F09C10034
:1003A00041088005100884001309C000400880053A
:1003B000110880040C0884000F088004410880059F
:1003C0000820100884001109C000400880051408A6
:1003D00080040C0884000F0880040F09C100410844
:1003E0008005100884001409C000400880050C082E
:1003F00084000F0880044108800508200F0880044D
:100400000F09C0004008800510088400140880040B
:100410000C0884000F08800440088005082010089C
:1004200084001409C000400880050C0884000F08EF
:1004300080040F09C10041088005100884001308DA
:100440001404C0001208C0041108C004400880044D
:100450000C0884000F088004410880050820013042
:1004600095000800442A803003138312A100572A04
:10047000C030A100572A9430A100572AD430A100DF
:10048000572A8030A100572A031383122108013A0A
:100490000319332A2108023A0319382A2108033A9A
:1004A00003193B2A2108043A03193E2A412A220350
:1004B000C0002108C0074008A1004008AC0022206D
:1004C0009501A4012408230784000008C000400807
:1004D0000319722A2408230784000008AA00AE200A
:1004E000A40A622A01309500080022300313831207
:1004F000A3002308AA00B7204008A1002308840015
:100500000008C0004008031D792A2108C000080027
:10051000031383121708A106160884001708003A6F
:10052000031D942A8010952A80141908AC009B2082
:10053000210803199B2A8010211880141908AC0087
:100540009B2021080319A42A8010A11880141908DF
:10055000AC009B2021080319AD2A801021198014BA
:100560001908AC009B2021080319B62A8010A11994
:1005700080141908AC009B2021080319BF2A8010A1
:10058000211A80141908AC009B2021080319C82ADD
:100590008010A11A80141908AC009B2021080319AF
:1005A000D12A8010211B80141908AC009B2021083F
:1005B0000319DA2A8010A11B80141908AC009B20B3
:1005C00080141908AC009B201A08800608004F30E0
:1005D000031383129B006B309C002E309D009E0104
:1005E0001B309F0008000313831221089900210883
:1005F0009800980C981316088400841780158010B2
:1006000084131708003A031D072B8014082B801051
:100610000800E72201308316850086010630960027
:100620006830A10097019A01F3220630A10007303B
:10063000A2000630A3000530A4000430A500063057
:10064000A600A7010130A8000230A9001A210C3031
:10065000AC0022200130A1000130A2001F08A3003D
:10066000322275224008A0004008FE3A031D3F2BAD
:1006700075224008A0004008AC002220422B200830
:10068000AA00AE20312B432BFF3FFF3FFF3FFF3F30
:02400E00F93F78
:00000001FF
